 wmstubber

 Timestamp is 66748569 (Thu Jun 20 19:39:21 2024)

 Preferred load address is 10000000

 Start         Length     Name                   Class
 0001:00000000 0000cfe0H .text                   CODE
 0001:0000cfe0 00000f14H .text$mn                CODE
 0002:00000000 000000f8H .idata$5                DATA
 0002:000000f8 00000004H .00cfg                  DATA
 0002:000000fc 00000004H .CRT$XCA                DATA
 0002:00000100 00000004H .CRT$XCZ                DATA
 0002:00000104 00000004H .CRT$XIA                DATA
 0002:00000108 00000004H .CRT$XIZ                DATA
 0002:0000010c 00000004H .CRT$XPA                DATA
 0002:00000110 00000004H .CRT$XPZ                DATA
 0002:00000114 00000004H .CRT$XTA                DATA
 0002:00000118 00000008H .CRT$XTZ                DATA
 0002:00000120 0000077cH .rdata                  DATA
 0002:0000089c 0000012cH .rdata$r                DATA
 0002:000009c8 00000258H .rdata$zzzdbg           DATA
 0002:00000c20 00000004H .rtc$IAA                DATA
 0002:00000c24 00000004H .rtc$IZZ                DATA
 0002:00000c28 00000004H .rtc$TAA                DATA
 0002:00000c2c 00000004H .rtc$TZZ                DATA
 0002:00000c30 00000110H .xdata$x                DATA
 0002:00000d40 00000060H .edata                  DATA
 0002:00000da0 00000078H .idata$2                DATA
 0002:00000e18 00000014H .idata$3                DATA
 0002:00000e2c 000000f8H .idata$4                DATA
 0002:00000f24 000004deH .idata$6                DATA
 0003:00000000 000008a0H .data                   DATA
 0003:000008a0 00000078H .data$r                 DATA
 0003:00000918 000008a0H .bss                    DATA
 0004:00000000 00000044H .gfids$y                DATA
 0005:00000000 000000a0H .rsrc$01                DATA
 0005:000000a0 00000588H .rsrc$02                DATA

  Address         Publics by Value              Rva+Base       Lib:Object

 0000:00000000       ___guard_longjmp_count     00000000     <absolute>
 0000:00000000       ___guard_fids_count        00000000     <absolute>
 0000:00000000       __except_list              00000000     <absolute>
 0000:00000000       ___safe_se_handler_table   00000000     <absolute>
 0000:00000000       ___guard_longjmp_table     00000000     <absolute>
 0000:00000000       ___dynamic_value_reloc_table 00000000     <absolute>
 0000:00000000       ___guard_iat_table         00000000     <absolute>
 0000:00000000       ___safe_se_handler_count   00000000     <absolute>
 0000:00000000       ___guard_iat_count         00000000     <absolute>
 0000:00000000       ___guard_fids_table        00000000     <absolute>
 0000:00000100       ___guard_flags             00000100     <absolute>
 0000:00009876       __ldused                   00009876     <absolute>
 0000:00000000       ___ImageBase               10000000     <linker-defined>
 0001:00000000       _WMCreateCertificate@4     10001000 f   wmstub:drmauth.obj
 0001:0000005c       ??0CWMAuthorizer@@QAE@XZ   1000105c f   wmstub:drmauth.obj
 0001:00000070       ??1CWMAuthorizer@@IAE@XZ   10001070 f   wmstub:drmauth.obj
 0001:0000008c       ?AddRef@CWMAuthorizer@@UAGKXZ 1000108c f   wmstub:drmauth.obj
 0001:0000009d       ?Release@CWMAuthorizer@@UAGKXZ 1000109d f   wmstub:drmauth.obj
 0001:000000c8       ?QueryInterface@CWMAuthorizer@@UAGJABU_GUID@@PAPAX@Z 100010c8 f   wmstub:drmauth.obj
 0001:00000112       ?GetCertCount@CWMAuthorizer@@UAGJPAK@Z 10001112 f   wmstub:drmauth.obj
 0001:00000141       ?GetCert@CWMAuthorizer@@UAGJKPAPAE@Z 10001141 f   wmstub:drmauth.obj
 0001:000001a9       ?GetSharedData@CWMAuthorizer@@UAGJKPBEPAEPAPAE@Z 100011a9 f   wmstub:drmauth.obj
 0001:000002f0       ?words_to_ecaffine@@YGHPBKPA_IPBUecurve_t@@@Z 100012f0 f   wmstub:pkcrypto.obj
 0001:00000520       ?i_PKinit@CDRMPKCrypto@@AAEJXZ 10001520 f   wmstub:pkcrypto.obj
 0001:00000540       ?PKinit@CDRMPKCrypto@@QAEJXZ 10001540 f   wmstub:pkcrypto.obj
 0001:00000570       ?i_CDRMPKCrypto@CDRMPKCrypto@@AAEXXZ 10001570 f   wmstub:pkcrypto.obj
 0001:00000740       ??0CDRMPKCrypto@@QAE@XZ    10001740 f   wmstub:pkcrypto.obj
 0001:00000790       ??1CDRMPKCrypto@@QAE@XZ    10001790 f   wmstub:pkcrypto.obj
 0001:000007f0       ?i_PKencrypt@CDRMPKCrypto@@AAEJPAUPUBKEY@@PAE1@Z 100017f0 f   wmstub:pkcrypto.obj
 0001:00000aa0       ?PKencrypt@CDRMPKCrypto@@QAEJPAUPUBKEY@@PAE1@Z 10001aa0 f   wmstub:pkcrypto.obj
 0001:00000ae0       ?i_PKdecrypt@CDRMPKCrypto@@AAEJPAUPRIVKEY@@PAE1@Z 10001ae0 f   wmstub:pkcrypto.obj
 0001:00000cc0       ?PKdecrypt@CDRMPKCrypto@@QAEJPAUPRIVKEY@@PAE1@Z 10001cc0 f   wmstub:pkcrypto.obj
 0001:00000d00       _Kadd@16                   10001d00 f   wmstub:field.obj
 0001:00000d70       _Kclear@12                 10001d70 f   wmstub:field.obj
 0001:00000da0       _Kcopy@16                  10001da0 f   wmstub:field.obj
 0001:00000dd0       _Kdiv@16                   10001dd0 f   wmstub:field.obj
 0001:00000e30       _Kequal@12                 10001e30 f   wmstub:field.obj
 0001:00000e80       _Kimmediate@12             10001e80 f   wmstub:field.obj
 0001:00000f10       _Kinitialize_prime@12      10001f10 f   wmstub:field.obj
 0001:00000f60       _Kinvert@12                10001f60 f   wmstub:field.obj
 0001:000010b0       _Kiszero@8                 100020b0 f   wmstub:field.obj
 0001:000010f0       _Kmul@16                   100020f0 f   wmstub:field.obj
 0001:00001160       _Kmuladd@20                10002160 f   wmstub:field.obj
 0001:000011d0       _Knegate@12                100021d0 f   wmstub:field.obj
 0001:00001220       _Ksqrt@12                  10002220 f   wmstub:field.obj
 0001:000012c0       _Ksub@16                   100022c0 f   wmstub:field.obj
 0001:00001330       _K2n_circular_shift@16     10002330 f   wmstub:field2n.obj
 0001:000013f0       _K2n_invert@12             100023f0 f   wmstub:field2n.obj
 0001:00001530       _K2n_multiply@16           10002530 f   wmstub:field2n.obj
 0001:000017e0       _K2_quad1@12               100027e0 f   wmstub:field2n.obj
 0001:000019a0       _create_modulus@16         100029a0 f   wmstub:modular.obj
 0001:00001ce0       _from_modular@12           10002ce0 f   wmstub:modular.obj
 0001:00001d40       _mod_add@16                10002d40 f   wmstub:modular.obj
 0001:00001dc0       _mod_mul@20                10002dc0 f   wmstub:modular.obj
 0001:00001eb0       _mod_mul_kara1@24          10002eb0 f   wmstub:modular.obj
 0001:00001f40       _mod_mul_kara@28           10002f40 f   wmstub:modular.obj
 0001:00001fa0       _mod_negate@12             10002fa0 f   wmstub:modular.obj
 0001:00001ff0       _mod_shift@16              10002ff0 f   wmstub:modular.obj
 0001:000021b0       _mod_sub@16                100031b0 f   wmstub:modular.obj
 0001:00002200       _modular_reduce@24         10003200 f   wmstub:modular.obj
 0001:00002a80       _to_modular@16             10003a80 f   wmstub:modular.obj
 0001:00002ba0       _mp_initialization@0       10003ba0 f   wmstub:mpglobal.obj
 0001:00002be0       _mp_alloc_temp@4           10003be0 f   wmstub:mpglobal.obj
 0001:00002c10       _mp_free_temp@4            10003c10 f   wmstub:mpglobal.obj
 0001:00002c30       _estimated_quotient_1@16   10003c30 f i wmstub:divide.obj
 0001:00002cb0       _div21@20                  10003cb0 f   wmstub:divide.obj
 0001:00002cf0       _divide@28                 10003cf0 f   wmstub:divide.obj
 0001:00002f50       _divide_immediate@20       10003f50 f   wmstub:divide.obj
 0001:00003130       _divide_precondition_1@12  10004130 f   wmstub:divide.obj
 0001:00003270       _ecaffine_exponentiation_tabular@28 10004270 f   wmstub:ecexpon.obj
 0001:000039d0       _ecaffine_table_construction@20 100049d0 f   wmstub:ecexpon.obj
 0001:00005500       _ecaffine_addition@20      10006500 f   wmstub:ecurve.obj
 0001:00005ac0       _ecaffine_is_infinite@8    10006ac0 f   wmstub:ecurve.obj
 0001:00005b80       _ecaffine_multiply_pm1@16  10006b80 f   wmstub:ecurve.obj
 0001:00005be0       _ecaffine_negate@12        10006be0 f   wmstub:ecurve.obj
 0001:00005c70       _ecaffine_on_curve@8       10006c70 f   wmstub:ecurve.obj
 0001:00005df0       _ecaffine_set_infinite@8   10006df0 f   wmstub:ecurve.obj
 0001:00005e60       _ec_initialize@16          10006e60 f   wmstub:ecurve.obj
 0001:00005f60       _random_digit_interval@8   10006f60 f   wmstub:mprand.obj
 0001:00005fc0       _random_mod@12             10006fc0 f   wmstub:mprand.obj
 0001:00006070       _random_mod_nonzero@12     10007070 f   wmstub:mprand.obj
 0001:000060f0       _accumulate@16             100070f0 f   wmstub:lowlev.obj
 0001:00006160       _add_diff@20               10007160 f   wmstub:lowlev.obj
 0001:00006220       _add_same@16               10007220 f   wmstub:lowlev.obj
 0001:00006290       _decumulate@16             10007290 f   wmstub:lowlev.obj
 0001:00006300       _multiply_immediate@16     10007300 f   wmstub:lowlev.obj
 0001:00006350       _multiply_low@16           10007350 f   wmstub:lowlev.obj
 0001:00006570       _sub_diff@20               10007570 f   wmstub:lowlev.obj
 0001:00006630       _sub_same@16               10007630 f   wmstub:lowlev.obj
 0001:000066a0       _add_full@20               100076a0 f   wmstub:mpmisc.obj
 0001:000066f0       _compare_diff@16           100076f0 f   wmstub:mpmisc.obj
 0001:00006790       _mp_longshift@16           10007790 f   wmstub:mpmisc.obj
 0001:00006830       _mp_shift@16               10007830 f   wmstub:mpmisc.obj
 0001:000069a0       _mp_significant_bit_count@8 100079a0 f   wmstub:mpmisc.obj
 0001:000069f0       _multiply@20               100079f0 f   wmstub:mpmisc.obj
 0001:00006aa0       _mp_gcdex@32               10007aa0 f   wmstub:mpgcdex.obj
 0001:00006eb0       _A_SHAInit@4               10007eb0 f   wmstub:sha.obj
 0001:00006ef0       _A_SHAUpdate@12            10007ef0 f   wmstub:sha.obj
 0001:00006fc0       _A_SHAUpdateNS@12          10007fc0 f   wmstub:sha.obj
 0001:00007090       _A_SHAFinalNS@8            10008090 f   wmstub:sha.obj
 0001:00007120       _mod_exp@20                10008120 f   wmstub:modexp.obj
 0001:00007690       _mod_exp_immediate@16      10008690 f   wmstub:modexp.obj
 0001:00007980       _GF2_extended_GCD@24       10008980 f   wmstub:field2p.obj
 0001:00007bc0       _GF2_mod_mul@20            10008bc0 f   wmstub:field2p.obj
 0001:00007d50       _gcdex_jacobi@16           10008d50 f   wmstub:gcdexjac.obj
 0001:000080b0       _random_bytes@8            100090b0 f   wmstub:randsupp.obj
 0001:000080d0       _mod_sqrt@12               100090d0 f   wmstub:modsqrt.obj
 0001:00008430       _padinfo_initialization@4  10009430 f   wmstub:kara.obj
 0001:000084c0       _find_padinfo@4            100094c0 f   wmstub:kara.obj
 0001:000084f0       _mul_kara@24               100094f0 f   wmstub:kara.obj
 0001:00008a70       _mul_kara_know_low@28      10009a70 f   wmstub:kara.obj
 0001:00008ef0       _to_kara@20                10009ef0 f   wmstub:kara.obj
 0001:00008fc0       _SHATransform@8            10009fc0 f   wmstub:shafast.obj
 0001:00009b2d       _SHATransform              1000ab2d f   wmstub:shafast.obj
 0001:00009b3d       _SHATransformNS@8          1000ab3d f   wmstub:shafast.obj
 0001:0000a682       _NewGenRandomEx@12         1000b682 f   wmstub:randlib.obj
 0001:0000a6f5       _NewGenRandom@16           1000b6f5 f   wmstub:randlib.obj
 0001:0000a750       _InitRand@8                1000b750 f   wmstub:randlib.obj
 0001:0000a7a7       _DeInitRand@8              1000b7a7 f   wmstub:randlib.obj
 0001:0000a7f5       _GenRandom@12              1000b7f5 f   wmstub:randlib.obj
 0001:0000a830       _RandomFillBuffer@8        1000b830 f   wmstub:randlib.obj
 0001:0000a906       _GatherRandomKey@16        1000b906 f   wmstub:randlib.obj
 0001:0000ad7d       _GatherRandomKeyFastUserMode@16 1000bd7d f   wmstub:randlib.obj
 0001:0000ae1f       _IsRNGWinNT@0              1000be1f f   wmstub:randlib.obj
 0001:0000af10       _mod_LucasUV@28            1000bf10 f   wmstub:lucas.obj
 0001:0000c460       _InitCircularHash@16       1000d460 f   wmstub:circhash.obj
 0001:0000c494       _GetCircularHashValue@12   1000d494 f   wmstub:circhash.obj
 0001:0000c4c0       _UpdateCircularHash@12     1000d4c0 f   wmstub:circhash.obj
 0001:0000c5ce       _ReadSeed@8                1000d5ce f   wmstub:seed.obj
 0001:0000c615       _WriteSeed@8               1000d615 f   wmstub:seed.obj
 0001:0000c658       _AccessSeed@8              1000d658 f   wmstub:seed.obj
 0001:0000c690       _rc4@12                    1000d690 f   wmstub:rc4fast.obj
 0001:0000c6f1       _rc4_key@12                1000d6f1 f   wmstub:rc4fast.obj
 0001:0000c75a       _rc4                       1000d75a f   wmstub:rc4fast.obj
 0001:0000c76f       _VeryLargeHashUpdate@12    1000d76f f   wmstub:vlhash.obj
 0001:0000c9e9       _GatherCPUSpecificCounters@8 1000d9e9 f   wmstub:cpu.obj
 0001:0000c9f0       _MD4Init@4                 1000d9f0 f   wmstub:md4ms.obj
 0001:0000ca20       _MD4Update@12              1000da20 f   wmstub:md4ms.obj
 0001:0000cb00       _MD4Final@4                1000db00 f   wmstub:md4ms.obj
 0001:0000cb60       _MD4Transform@8            1000db60 f   wmstub:md4fast.obj
 0001:0000cfc9       _MD4Transform              1000dfc9 f   wmstub:md4fast.obj
 0001:0000cfe0       _DllMain@12                1000dfe0 f   wmstubber.obj
 0001:0000cff0       _get_wmcreatecertificate_func 1000dff0 f   wmstubber.obj
 0001:0000d305       __DllMainCRTStartup@12     1000e305 f   MSVCRT:dll_dllmain.obj
 0001:0000d328       ??2@YAPAXI@Z               1000e328 f   MSVCRT:new_scalar.obj
 0001:0000d35b       ??3@YAXPAX@Z               1000e35b f   MSVCRT:delete_scalar.obj
 0001:0000d360       __aulldiv                  1000e360 f   MSVCRT:ulldiv.obj
 0001:0000d3d0       __alloca_probe             1000e3d0 f   MSVCRT:chkstk.obj
 0001:0000d3d0       __chkstk                   1000e3d0 f   MSVCRT:chkstk.obj
 0001:0000d400       __allmul                   1000e400 f   MSVCRT:llmul.obj
 0001:0000d484       ___scrt_acquire_startup_lock 1000e484 f   MSVCRT:utility.obj
 0001:0000d4b9       ___scrt_dllmain_after_initialize_c 1000e4b9 f   MSVCRT:utility.obj
 0001:0000d4e4       ___scrt_dllmain_before_initialize_c 1000e4e4 f   MSVCRT:utility.obj
 0001:0000d4f2       ___scrt_dllmain_crt_thread_attach 1000e4f2 f   MSVCRT:utility.obj
 0001:0000d511       ___scrt_dllmain_crt_thread_detach 1000e511 f   MSVCRT:utility.obj
 0001:0000d51e       ___scrt_dllmain_exception_filter 1000e51e f   MSVCRT:utility.obj
 0001:0000d551       ___scrt_dllmain_uninitialize_c 1000e551 f   MSVCRT:utility.obj
 0001:0000d574       ___scrt_dllmain_uninitialize_critical 1000e574 f   MSVCRT:utility.obj
 0001:0000d581       ___scrt_initialize_crt     1000e581 f   MSVCRT:utility.obj
 0001:0000d5ba       ___scrt_initialize_onexit_tables 1000e5ba f   MSVCRT:utility.obj
 0001:0000d651       ___scrt_is_nonwritable_in_current_image 1000e651 f   MSVCRT:utility.obj
 0001:0000d6db       ___scrt_release_startup_lock 1000e6db f   MSVCRT:utility.obj
 0001:0000d6f8       ___scrt_uninitialize_crt   1000e6f8 f   MSVCRT:utility.obj
 0001:0000d720       __onexit                   1000e720 f   MSVCRT:utility.obj
 0001:0000d75b       _atexit                    1000e75b f   MSVCRT:utility.obj
 0001:0000d770       ___security_init_cookie    1000e770 f   MSVCRT:gs_support.obj
 0001:0000d80c       ?__scrt_initialize_type_info@@YAXXZ 1000e80c f   MSVCRT:tncleanup.obj
 0001:0000d818       ?__scrt_uninitialize_type_info@@YAXXZ 1000e818 f   MSVCRT:tncleanup.obj
 0001:0000d824       ___local_stdio_printf_options 1000e824 f i MSVCRT:default_local_stdio_options.obj
 0001:0000d82a       ___local_stdio_scanf_options 1000e82a f i MSVCRT:default_local_stdio_options.obj
 0001:0000d830       ___scrt_initialize_default_local_stdio_options 1000e830 f   MSVCRT:default_local_stdio_options.obj
 0001:0000d84d       ___scrt_get_dyn_tls_init_callback 1000e84d f   MSVCRT:dyn_tls_init.obj
 0001:0000d853       ___scrt_fastfail           1000e853 f   MSVCRT:utility_desktop.obj
 0001:0000d96e       __RTC_Initialize           1000e96e f   MSVCRT:_initsect_.obj
 0001:0000d999       __RTC_Terminate            1000e999 f   MSVCRT:_initsect_.obj
 0001:0000d9c4       @_guard_check_icall@4      1000e9c4 f i MSVCRT:checkcfg.obj
 0001:0000d9d0       __SEH_prolog4              1000e9d0 f   MSVCRT:_sehprolg4_.obj
 0001:0000da16       __SEH_epilog4              1000ea16 f   MSVCRT:_sehprolg4_.obj
 0001:0000da2b       __except_handler4          1000ea2b f   MSVCRT:_chandler4gs_.obj
 0001:0000da4e       ??0bad_alloc@std@@QAE@ABV01@@Z 1000ea4e f i MSVCRT:throw_bad_alloc.obj
 0001:0000da69       ??0bad_alloc@std@@QAE@XZ   1000ea69 f i MSVCRT:throw_bad_alloc.obj
 0001:0000da81       ??0bad_array_new_length@std@@QAE@ABV01@@Z 1000ea81 f i MSVCRT:throw_bad_alloc.obj
 0001:0000da9c       ??0bad_array_new_length@std@@QAE@XZ 1000ea9c f i MSVCRT:throw_bad_alloc.obj
 0001:0000dab4       ??0exception@std@@QAE@ABV01@@Z 1000eab4 f i MSVCRT:throw_bad_alloc.obj
 0001:0000dae0       ??1bad_array_new_length@std@@UAE@XZ 1000eae0 f i MSVCRT:throw_bad_alloc.obj
 0001:0000dae0       ??1bad_alloc@std@@UAE@XZ   1000eae0 f i MSVCRT:throw_bad_alloc.obj
 0001:0000daf1       ??_Ebad_array_new_length@std@@UAEPAXI@Z 1000eaf1 f i MSVCRT:throw_bad_alloc.obj
 0001:0000daf1       ??_Gbad_alloc@std@@UAEPAXI@Z 1000eaf1 f i MSVCRT:throw_bad_alloc.obj
 0001:0000daf1       ??_Ebad_alloc@std@@UAEPAXI@Z 1000eaf1 f i MSVCRT:throw_bad_alloc.obj
 0001:0000daf1       ??_Gexception@std@@UAEPAXI@Z 1000eaf1 f i MSVCRT:throw_bad_alloc.obj
 0001:0000daf1       ??_Gbad_array_new_length@std@@UAEPAXI@Z 1000eaf1 f i MSVCRT:throw_bad_alloc.obj
 0001:0000daf1       ??_Eexception@std@@UAEPAXI@Z 1000eaf1 f i MSVCRT:throw_bad_alloc.obj
 0001:0000db1e       ?__scrt_throw_std_bad_alloc@@YAXXZ 1000eb1e f   MSVCRT:throw_bad_alloc.obj
 0001:0000db3b       ?__scrt_throw_std_bad_array_new_length@@YAXXZ 1000eb3b f   MSVCRT:throw_bad_alloc.obj
 0001:0000db58       ?what@exception@std@@UBEPBDXZ 1000eb58 f i MSVCRT:throw_bad_alloc.obj
 0001:0000db65       ___isa_available_init      1000eb65 f   MSVCRT:_cpu_disp_.obj
 0001:0000dcff       __get_startup_argv_mode    1000ecff f   MSVCRT:argv_mode.obj
 0001:0000dd03       ___scrt_is_ucrt_dll_in_use 1000ed03 f   MSVCRT:ucrt_detection.obj
 0001:0000dd0f       @_guard_check_icall_nop@4  1000ed0f f i MSVCRT:guard_support.obj
 0001:0000dd10       @__security_check_cookie@4 1000ed10 f   MSVCRT:_secchk_.obj
 0001:0000dd21       ??3@YAXPAXI@Z              1000ed21 f   MSVCRT:delete_scalar_size.obj
 0001:0000dd2f       ??_Etype_info@@UAEPAXI@Z   1000ed2f f i MSVCRT:std_type_info_static.obj
 0001:0000dd2f       ??_Gtype_info@@UAEPAXI@Z   1000ed2f f i MSVCRT:std_type_info_static.obj
 0001:0000dd52       ___raise_securityfailure   1000ed52 f   MSVCRT:gs_report.obj
 0001:0000dd7a       ___report_gsfailure        1000ed7a f   MSVCRT:gs_report.obj
 0001:0000de76       ___std_type_info_destroy_list 1000ee76 f   vcruntime:VCRUNTIME140.dll
 0001:0000de7c       _memset                    1000ee7c f   vcruntime:VCRUNTIME140.dll
 0001:0000de82       __except_handler4_common   1000ee82 f   vcruntime:VCRUNTIME140.dll
 0001:0000de88       ___std_exception_copy      1000ee88 f   vcruntime:VCRUNTIME140.dll
 0001:0000de8e       ___std_exception_destroy   1000ee8e f   vcruntime:VCRUNTIME140.dll
 0001:0000de94       __CxxThrowException@8      1000ee94 f   vcruntime:VCRUNTIME140.dll
 0001:0000de9a       __initterm                 1000ee9a f   ucrt:api-ms-win-crt-runtime-l1-1-0.dll
 0001:0000dea0       __initterm_e               1000eea0 f   ucrt:api-ms-win-crt-runtime-l1-1-0.dll
 0001:0000dea6       __callnewh                 1000eea6 f   ucrt:api-ms-win-crt-heap-l1-1-0.dll
 0001:0000deac       _malloc                    1000eeac f   ucrt:api-ms-win-crt-heap-l1-1-0.dll
 0001:0000deb2       _free                      1000eeb2 f   ucrt:api-ms-win-crt-heap-l1-1-0.dll
 0001:0000deb8       __seh_filter_dll           1000eeb8 f   ucrt:api-ms-win-crt-runtime-l1-1-0.dll
 0001:0000debe       __configure_narrow_argv    1000eebe f   ucrt:api-ms-win-crt-runtime-l1-1-0.dll
 0001:0000dec4       __initialize_narrow_environment 1000eec4 f   ucrt:api-ms-win-crt-runtime-l1-1-0.dll
 0001:0000deca       __initialize_onexit_table  1000eeca f   ucrt:api-ms-win-crt-runtime-l1-1-0.dll
 0001:0000ded0       __register_onexit_function 1000eed0 f   ucrt:api-ms-win-crt-runtime-l1-1-0.dll
 0001:0000ded6       __execute_onexit_table     1000eed6 f   ucrt:api-ms-win-crt-runtime-l1-1-0.dll
 0001:0000dedc       __crt_atexit               1000eedc f   ucrt:api-ms-win-crt-runtime-l1-1-0.dll
 0001:0000dee2       __cexit                    1000eee2 f   ucrt:api-ms-win-crt-runtime-l1-1-0.dll
 0001:0000dee8       _IsProcessorFeaturePresent@4 1000eee8 f   kernel32:KERNEL32.dll
 0001:0000deee       ___acrt_uninitialize_critical 1000eeee f   MSVCRT:ucrt_stubs.obj
 0001:0000deee       ___scrt_stub_for_acrt_thread_attach 1000eeee f   MSVCRT:ucrt_stubs.obj
 0001:0000deee       ___vcrt_initialize         1000eeee f   MSVCRT:ucrt_stubs.obj
 0001:0000deee       ___scrt_stub_for_acrt_uninitialize_critical 1000eeee f   MSVCRT:ucrt_stubs.obj
 0001:0000deee       ___acrt_initialize         1000eeee f   MSVCRT:ucrt_stubs.obj
 0001:0000deee       ___acrt_thread_attach      1000eeee f   MSVCRT:ucrt_stubs.obj
 0001:0000deee       ___vcrt_thread_attach      1000eeee f   MSVCRT:ucrt_stubs.obj
 0001:0000deee       ___vcrt_uninitialize       1000eeee f   MSVCRT:ucrt_stubs.obj
 0001:0000deee       ___scrt_stub_for_acrt_thread_detach 1000eeee f   MSVCRT:ucrt_stubs.obj
 0001:0000deee       ___acrt_thread_detach      1000eeee f   MSVCRT:ucrt_stubs.obj
 0001:0000deee       ___scrt_stub_for_acrt_uninitialize 1000eeee f   MSVCRT:ucrt_stubs.obj
 0001:0000deee       ___vcrt_uninitialize_critical 1000eeee f   MSVCRT:ucrt_stubs.obj
 0001:0000deee       ___scrt_stub_for_acrt_initialize 1000eeee f   MSVCRT:ucrt_stubs.obj
 0001:0000deee       ___vcrt_thread_detach      1000eeee f   MSVCRT:ucrt_stubs.obj
 0001:0000deee       ___acrt_uninitialize       1000eeee f   MSVCRT:ucrt_stubs.obj
 0001:0000def1       __is_c_termination_complete 1000eef1 f   MSVCRT:ucrt_stubs.obj
 0001:0000def1       ___scrt_stub_for_is_c_termination_complete 1000eef1 f   MSVCRT:ucrt_stubs.obj
 0002:00000000       __imp__GetUserNameA@8      1000f000     advapi32:ADVAPI32.dll
 0002:00000004       __imp__RegQueryValueExA@24 1000f004     advapi32:ADVAPI32.dll
 0002:00000008       __imp__RegSetValueExA@24   1000f008     advapi32:ADVAPI32.dll
 0002:0000000c       __imp__RegCreateKeyExA@36  1000f00c     advapi32:ADVAPI32.dll
 0002:00000010       __imp__RegCloseKey@4       1000f010     advapi32:ADVAPI32.dll
 0002:00000014       \177ADVAPI32_NULL_THUNK_DATA 1000f014     advapi32:ADVAPI32.dll
 0002:00000018       __imp__GlobalMemoryStatus@4 1000f018     kernel32:KERNEL32.dll
 0002:0000001c       __imp__GetTickCount@0      1000f01c     kernel32:KERNEL32.dll
 0002:00000020       __imp__GetCurrentThreadId@0 1000f020     kernel32:KERNEL32.dll
 0002:00000024       __imp__GetCurrentProcessId@0 1000f024     kernel32:KERNEL32.dll
 0002:00000028       __imp__CloseHandle@4       1000f028     kernel32:KERNEL32.dll
 0002:0000002c       __imp__QueryPerformanceCounter@4 1000f02c     kernel32:KERNEL32.dll
 0002:00000030       __imp__GetLocalTime@4      1000f030     kernel32:KERNEL32.dll
 0002:00000034       __imp__LocalAlloc@8        1000f034     kernel32:KERNEL32.dll
 0002:00000038       __imp__TerminateProcess@8  1000f038     kernel32:KERNEL32.dll
 0002:0000003c       __imp__GetCurrentProcess@0 1000f03c     kernel32:KERNEL32.dll
 0002:00000040       __imp__IsProcessorFeaturePresent@4 1000f040     kernel32:KERNEL32.dll
 0002:00000044       __imp__SetUnhandledExceptionFilter@4 1000f044     kernel32:KERNEL32.dll
 0002:00000048       __imp__UnhandledExceptionFilter@4 1000f048     kernel32:KERNEL32.dll
 0002:0000004c       __imp__IsDebuggerPresent@0 1000f04c     kernel32:KERNEL32.dll
 0002:00000050       __imp__InitializeSListHead@4 1000f050     kernel32:KERNEL32.dll
 0002:00000054       __imp__GetSystemTimeAsFileTime@4 1000f054     kernel32:KERNEL32.dll
 0002:00000058       __imp__GetVersionExA@4     1000f058     kernel32:KERNEL32.dll
 0002:0000005c       __imp__GetModuleHandleW@4  1000f05c     kernel32:KERNEL32.dll
 0002:00000060       __imp__GetProcAddress@8    1000f060     kernel32:KERNEL32.dll
 0002:00000064       __imp__LoadLibraryA@4      1000f064     kernel32:KERNEL32.dll
 0002:00000068       __imp__InterlockedIncrement@4 1000f068     kernel32:KERNEL32.dll
 0002:0000006c       __imp__InterlockedDecrement@4 1000f06c     kernel32:KERNEL32.dll
 0002:00000070       __imp__LeaveCriticalSection@4 1000f070     kernel32:KERNEL32.dll
 0002:00000074       __imp__EnterCriticalSection@4 1000f074     kernel32:KERNEL32.dll
 0002:00000078       __imp__InitializeCriticalSection@4 1000f078     kernel32:KERNEL32.dll
 0002:0000007c       __imp__GetSystemInfo@4     1000f07c     kernel32:KERNEL32.dll
 0002:00000080       __imp__GetDiskFreeSpaceA@20 1000f080     kernel32:KERNEL32.dll
 0002:00000084       __imp__LocalFree@4         1000f084     kernel32:KERNEL32.dll
 0002:00000088       __imp__GetComputerNameA@8  1000f088     kernel32:KERNEL32.dll
 0002:0000008c       __imp__DeviceIoControl@32  1000f08c     kernel32:KERNEL32.dll
 0002:00000090       \177KERNEL32_NULL_THUNK_DATA 1000f090     kernel32:KERNEL32.dll
 0002:00000094       __imp___CxxThrowException@8 1000f094     vcruntime:VCRUNTIME140.dll
 0002:00000098       __imp____std_exception_destroy 1000f098     vcruntime:VCRUNTIME140.dll
 0002:0000009c       __imp____std_exception_copy 1000f09c     vcruntime:VCRUNTIME140.dll
 0002:000000a0       __imp___except_handler4_common 1000f0a0     vcruntime:VCRUNTIME140.dll
 0002:000000a4       __imp__memset              1000f0a4     vcruntime:VCRUNTIME140.dll
 0002:000000a8       __imp____std_type_info_destroy_list 1000f0a8     vcruntime:VCRUNTIME140.dll
 0002:000000ac       \177VCRUNTIME140_NULL_THUNK_DATA 1000f0ac     vcruntime:VCRUNTIME140.dll
 0002:000000b0       __imp__free                1000f0b0     ucrt:api-ms-win-crt-heap-l1-1-0.dll
 0002:000000b4       __imp__malloc              1000f0b4     ucrt:api-ms-win-crt-heap-l1-1-0.dll
 0002:000000b8       __imp___callnewh           1000f0b8     ucrt:api-ms-win-crt-heap-l1-1-0.dll
 0002:000000bc       \177api-ms-win-crt-heap-l1-1-0_NULL_THUNK_DATA 1000f0bc     ucrt:api-ms-win-crt-heap-l1-1-0.dll
 0002:000000c0       __imp___execute_onexit_table 1000f0c0     ucrt:api-ms-win-crt-runtime-l1-1-0.dll
 0002:000000c4       __imp___register_onexit_function 1000f0c4     ucrt:api-ms-win-crt-runtime-l1-1-0.dll
 0002:000000c8       __imp___initialize_onexit_table 1000f0c8     ucrt:api-ms-win-crt-runtime-l1-1-0.dll
 0002:000000cc       __imp___crt_atexit         1000f0cc     ucrt:api-ms-win-crt-runtime-l1-1-0.dll
 0002:000000d0       __imp___configure_narrow_argv 1000f0d0     ucrt:api-ms-win-crt-runtime-l1-1-0.dll
 0002:000000d4       __imp___seh_filter_dll     1000f0d4     ucrt:api-ms-win-crt-runtime-l1-1-0.dll
 0002:000000d8       __imp___cexit              1000f0d8     ucrt:api-ms-win-crt-runtime-l1-1-0.dll
 0002:000000dc       __imp___initterm_e         1000f0dc     ucrt:api-ms-win-crt-runtime-l1-1-0.dll
 0002:000000e0       __imp___initterm           1000f0e0     ucrt:api-ms-win-crt-runtime-l1-1-0.dll
 0002:000000e4       __imp___initialize_narrow_environment 1000f0e4     ucrt:api-ms-win-crt-runtime-l1-1-0.dll
 0002:000000e8       \177api-ms-win-crt-runtime-l1-1-0_NULL_THUNK_DATA 1000f0e8     ucrt:api-ms-win-crt-runtime-l1-1-0.dll
 0002:000000ec       __imp__CoTaskMemAlloc@4    1000f0ec     ole32:ole32.dll
 0002:000000f0       __imp__CoTaskMemFree@4     1000f0f0     ole32:ole32.dll
 0002:000000f4       \177ole32_NULL_THUNK_DATA  1000f0f4     ole32:ole32.dll
 0002:000000f8       ___guard_check_icall_fptr  1000f0f8     MSVCRT:guard_support.obj
 0002:000000fc       ___xc_a                    1000f0fc     MSVCRT:initializers.obj
 0002:00000100       ___xc_z                    1000f100     MSVCRT:initializers.obj
 0002:00000104       ___xi_a                    1000f104     MSVCRT:initializers.obj
 0002:00000108       ___xi_z                    1000f108     MSVCRT:initializers.obj
 0002:0000010c       ___xp_a                    1000f10c     MSVCRT:initializers.obj
 0002:00000110       ___xp_z                    1000f110     MSVCRT:initializers.obj
 0002:00000114       ___xt_a                    1000f114     MSVCRT:initializers.obj
 0002:00000118       ___xt_z                    1000f118     MSVCRT:initializers.obj
 0002:000005a0       _IID_IWMAuthorizer         1000f5a0     wmstub:drmauth.obj
 0002:000005b0       ??_7CWMAuthorizer@@6B@     1000f5b0     wmstub:drmauth.obj
 0002:00000640       _POWER3                    1000f640     wmstub:mpglobal.obj
 0002:00000688       ??_C@_1BO@IBIA@?$AA?2?$AAD?$AAe?$AAv?$AAi?$AAc?$AAe?$AA?2?$AAK?$AAs?$AAe?$AAc?$AAD?$AAD?$AA?$AA@ 1000f688     wmstub:randlib.obj
 0002:000006a8       ??_C@_0P@PLIF@GetMessageTime?$AA@ 1000f6a8     wmstub:randlib.obj
 0002:000006b8       ??_C@_0N@OKFA@GetCursorPos?$AA@ 1000f6b8     wmstub:randlib.obj
 0002:000006c8       ??_C@_0L@HKL@user32?4dll?$AA@ 1000f6c8     wmstub:randlib.obj
 0002:000006d4       ??_C@_0BF@LGHK@RtlInitUnicodeString?$AA@ 1000f6d4     wmstub:randlib.obj
 0002:000006ec       ??_C@_0L@EOEO@NtOpenFile?$AA@ 1000f6ec     wmstub:randlib.obj
 0002:000006f8       ??_C@_0BJ@FIKA@NtQuerySystemInformation?$AA@ 1000f6f8     wmstub:randlib.obj
 0002:00000714       ??_C@_1BE@GHKF@?$AAn?$AAt?$AAd?$AAl?$AAl?$AA?4?$AAd?$AAl?$AAl?$AA?$AA@ 1000f714     wmstub:randlib.obj
 0002:00000728       ??_C@_04NNOK@Seed?$AA@     1000f728     wmstub:seed.obj
 0002:00000730       ??_C@_0CE@PBOJ@SOFTWARE?2Microsoft?2Cryptography?2@ 1000f730     wmstub:seed.obj
 0002:00000798       __pDefaultRawDllMain       1000f798     MSVCRT:dll_dllmain.obj
 0002:00000798       __pRawDllMain              1000f798     MSVCRT:dll_dllmain.obj
 0002:000007a0       ??_7exception@std@@6B@     1000f7a0     MSVCRT:throw_bad_alloc.obj
 0002:000007a8       ??_C@_0BC@EOODALEL@Unknown?5exception?$AA@ 1000f7a8     MSVCRT:throw_bad_alloc.obj
 0002:000007c0       ??_7bad_alloc@std@@6B@     1000f7c0     MSVCRT:throw_bad_alloc.obj
 0002:000007c8       ??_C@_0P@GHFPNOJB@bad?5allocation?$AA@ 1000f7c8     MSVCRT:throw_bad_alloc.obj
 0002:000007dc       ??_7bad_array_new_length@std@@6B@ 1000f7dc     MSVCRT:throw_bad_alloc.obj
 0002:000007e4       ??_C@_0BF@KINCDENJ@bad?5array?5new?5length?$AA@ 1000f7e4     MSVCRT:throw_bad_alloc.obj
 0002:00000800       ??_7type_info@@6B@         1000f800     MSVCRT:std_type_info_static.obj
 0002:0000080c       _IID_IUnknown              1000f80c     uuid:unknwn_i.obj
 0002:00000840       __load_config_used         1000f840     MSVCRT:loadcfg.obj
 0002:0000089c       ??_R4exception@std@@6B@    1000f89c     MSVCRT:throw_bad_alloc.obj
 0002:000008b0       ??_R3exception@std@@8      1000f8b0     MSVCRT:throw_bad_alloc.obj
 0002:000008c0       ??_R2exception@std@@8      1000f8c0     MSVCRT:throw_bad_alloc.obj
 0002:000008c8       ??_R1A@?0A@EA@exception@std@@8 1000f8c8     MSVCRT:throw_bad_alloc.obj
 0002:000008e4       ??_R4bad_alloc@std@@6B@    1000f8e4     MSVCRT:throw_bad_alloc.obj
 0002:000008f8       ??_R3bad_alloc@std@@8      1000f8f8     MSVCRT:throw_bad_alloc.obj
 0002:00000908       ??_R2bad_alloc@std@@8      1000f908     MSVCRT:throw_bad_alloc.obj
 0002:00000914       ??_R1A@?0A@EA@bad_alloc@std@@8 1000f914     MSVCRT:throw_bad_alloc.obj
 0002:00000930       ??_R4bad_array_new_length@std@@6B@ 1000f930     MSVCRT:throw_bad_alloc.obj
 0002:00000944       ??_R3bad_array_new_length@std@@8 1000f944     MSVCRT:throw_bad_alloc.obj
 0002:00000954       ??_R2bad_array_new_length@std@@8 1000f954     MSVCRT:throw_bad_alloc.obj
 0002:00000964       ??_R1A@?0A@EA@bad_array_new_length@std@@8 1000f964     MSVCRT:throw_bad_alloc.obj
 0002:00000980       ??_R4type_info@@6B@        1000f980     MSVCRT:std_type_info_static.obj
 0002:00000994       ??_R3type_info@@8          1000f994     MSVCRT:std_type_info_static.obj
 0002:000009a4       ??_R2type_info@@8          1000f9a4     MSVCRT:std_type_info_static.obj
 0002:000009ac       ??_R1A@?0A@EA@type_info@@8 1000f9ac     MSVCRT:std_type_info_static.obj
 0002:00000c20       ___rtc_iaa                 1000fc20     MSVCRT:_initsect_.obj
 0002:00000c24       ___rtc_izz                 1000fc24     MSVCRT:_initsect_.obj
 0002:00000c28       ___rtc_taa                 1000fc28     MSVCRT:_initsect_.obj
 0002:00000c2c       ___rtc_tzz                 1000fc2c     MSVCRT:_initsect_.obj
 0002:00000cac       __TI2?AVbad_alloc@std@@    1000fcac     MSVCRT:throw_bad_alloc.obj
 0002:00000cbc       __CTA2?AVbad_alloc@std@@   1000fcbc     MSVCRT:throw_bad_alloc.obj
 0002:00000cc8       __CT??_R0?AVbad_alloc@std@@@8??0bad_alloc@std@@QAE@ABV01@@Z12 1000fcc8     MSVCRT:throw_bad_alloc.obj
 0002:00000ce4       __CT??_R0?AVexception@std@@@8??0exception@std@@QAE@ABV01@@Z12 1000fce4     MSVCRT:throw_bad_alloc.obj
 0002:00000d00       __TI3?AVbad_array_new_length@std@@ 1000fd00     MSVCRT:throw_bad_alloc.obj
 0002:00000d10       __CTA3?AVbad_array_new_length@std@@ 1000fd10     MSVCRT:throw_bad_alloc.obj
 0002:00000d20       __CT??_R0?AVbad_array_new_length@std@@@8??0bad_array_new_length@std@@QAE@ABV01@@Z12 1000fd20     MSVCRT:throw_bad_alloc.obj
 0002:00000da0       __IMPORT_DESCRIPTOR_VCRUNTIME140 1000fda0     vcruntime:VCRUNTIME140.dll
 0002:00000db4       __IMPORT_DESCRIPTOR_api-ms-win-crt-runtime-l1-1-0 1000fdb4     ucrt:api-ms-win-crt-runtime-l1-1-0.dll
 0002:00000dc8       __IMPORT_DESCRIPTOR_api-ms-win-crt-heap-l1-1-0 1000fdc8     ucrt:api-ms-win-crt-heap-l1-1-0.dll
 0002:00000ddc       __IMPORT_DESCRIPTOR_KERNEL32 1000fddc     kernel32:KERNEL32.dll
 0002:00000df0       __IMPORT_DESCRIPTOR_ADVAPI32 1000fdf0     advapi32:ADVAPI32.dll
 0002:00000e04       __IMPORT_DESCRIPTOR_ole32  1000fe04     ole32:ole32.dll
 0002:00000e18       __NULL_IMPORT_DESCRIPTOR   1000fe18     vcruntime:VCRUNTIME140.dll
 0003:000000b8       ??_C@_1CC@JCME@?$AA_?$AAS?$AAO?$AAU?$AAR?$AAC?$AAE?$AAF?$AAO?$AAR?$AAM?$AAA?$AAT?$AAT?$AAA?$AAG?$AA?$AA@ 100110b8     wmstub:drmauth.obj
 0003:000000dc       ??_C@_1CA@NJFP@?$AAD?$AAe?$AAi?$AAn?$AAt?$AAe?$AAr?$AAl?$AAa?$AAc?$AAe?$AAM?$AAo?$AAd?$AAe?$AA?$AA@ 100110dc     wmstub:drmauth.obj
 0003:000000fc       ??_C@_1CC@FOMH@?$AAD?$AAe?$AAl?$AAi?$AAv?$AAe?$AAr?$AAO?$AAn?$AAR?$AAe?$AAc?$AAe?$AAi?$AAv?$AAe?$AA?$AA@ 100110fc     wmstub:drmauth.obj
 0003:00000120       ??_C@_1CA@NFFK@?$AAS?$AAo?$AAf?$AAt?$AAw?$AAa?$AAr?$AAe?$AAS?$AAc?$AAa?$AAl?$AAi?$AAn?$AAg?$AA?$AA@ 10011120     wmstub:drmauth.obj
 0003:00000140       ??_C@_1CG@MJPE@?$AAS?$AAi?$AAn?$AAg?$AAl?$AAe?$AAO?$AAu?$AAt?$AAp?$AAu?$AAt?$AAB?$AAu?$AAf?$AAf?$AAe?$AAr?$AA?$AA@ 10011140     wmstub:drmauth.obj
 0003:00000168       ??_C@_1CC@NLDH@?$AAJ?$AAu?$AAs?$AAt?$AAI?$AAn?$AAT?$AAi?$AAm?$AAe?$AAD?$AAe?$AAc?$AAo?$AAd?$AAe?$AA?$AA@ 10011168     wmstub:drmauth.obj
 0003:0000018c       ??_C@_1CE@EKBE@?$AAE?$AAa?$AAr?$AAl?$AAy?$AAD?$AAa?$AAt?$AAa?$AAD?$AAe?$AAl?$AAi?$AAv?$AAe?$AAr?$AAy?$AA?$AA@ 1001118c     wmstub:drmauth.obj
 0003:000001b0       ??_C@_1CA@KGHO@?$AAN?$AAS?$AAC?$AA_?$AAD?$AAe?$AAs?$AAc?$AAr?$AAi?$AAp?$AAt?$AAi?$AAo?$AAn?$AA?$AA@ 100111b0     wmstub:drmauth.obj
 0003:000001d0       ??_C@_1BE@LDNB@?$AAN?$AAS?$AAC?$AA_?$AAE?$AAm?$AAa?$AAi?$AAl?$AA?$AA@ 100111d0     wmstub:drmauth.obj
 0003:000001e4       ??_C@_1BE@KBHM@?$AAN?$AAS?$AAC?$AA_?$AAP?$AAh?$AAo?$AAn?$AAe?$AA?$AA@ 100111e4     wmstub:drmauth.obj
 0003:000001f8       ??_C@_1BI@MCHF@?$AAN?$AAS?$AAC?$AA_?$AAA?$AAd?$AAd?$AAr?$AAe?$AAs?$AAs?$AA?$AA@ 100111f8     wmstub:drmauth.obj
 0003:00000210       ??_C@_1BC@JDLO@?$AAN?$AAS?$AAC?$AA_?$AAN?$AAa?$AAm?$AAe?$AA?$AA@ 10011210     wmstub:drmauth.obj
 0003:00000224       ??_C@_1BK@JIPJ@?$AAC?$AAo?$AAp?$AAy?$AAr?$AAi?$AAg?$AAh?$AAt?$AAU?$AAR?$AAL?$AA?$AA@ 10011224     wmstub:drmauth.obj
 0003:00000240       ??_C@_1BO@HME@?$AAB?$AAa?$AAn?$AAn?$AAe?$AAr?$AAI?$AAm?$AAa?$AAg?$AAe?$AAU?$AAR?$AAL?$AA?$AA@ 10011240     wmstub:drmauth.obj
 0003:00000260       ??_C@_1CA@HBBE@?$AAB?$AAa?$AAn?$AAn?$AAe?$AAr?$AAI?$AAm?$AAa?$AAg?$AAe?$AAD?$AAa?$AAt?$AAa?$AA?$AA@ 10011260     wmstub:drmauth.obj
 0003:00000280       ??_C@_1CA@KO@?$AAB?$AAa?$AAn?$AAn?$AAe?$AAr?$AAI?$AAm?$AAa?$AAg?$AAe?$AAT?$AAy?$AAp?$AAe?$AA?$AA@ 10011280     wmstub:drmauth.obj
 0003:000002a0       ??_C@_1BA@MIKK@?$AAW?$AAM?$AA?1?$AAM?$AAC?$AAD?$AAI?$AA?$AA@ 100112a0     wmstub:drmauth.obj
 0003:000002b0       ??_C@_1BG@NMNO@?$AAW?$AAM?$AA?1?$AAG?$AAe?$AAn?$AAr?$AAe?$AAI?$AAD?$AA?$AA@ 100112b0     wmstub:drmauth.obj
 0003:000002c8       ??_C@_1BA@PBOK@?$AAW?$AAM?$AA?1?$AAY?$AAe?$AAa?$AAr?$AA?$AA@ 100112c8     wmstub:drmauth.obj
 0003:000002d8       ??_C@_1BC@LDIK@?$AAW?$AAM?$AA?1?$AAG?$AAe?$AAn?$AAr?$AAe?$AA?$AA@ 100112d8     wmstub:drmauth.obj
 0003:000002ec       ??_C@_1CC@BANO@?$AAW?$AAM?$AA?1?$AAA?$AAl?$AAb?$AAu?$AAm?$AAC?$AAo?$AAv?$AAe?$AAr?$AAU?$AAR?$AAL?$AA?$AA@ 100112ec     wmstub:drmauth.obj
 0003:00000310       ??_C@_1CA@BPCC@?$AAW?$AAM?$AA?1?$AAP?$AAr?$AAo?$AAm?$AAo?$AAt?$AAi?$AAo?$AAn?$AAU?$AAR?$AAL?$AA?$AA@ 10011310     wmstub:drmauth.obj
 0003:00000330       ??_C@_1BC@CMGL@?$AAW?$AAM?$AA?1?$AAT?$AAr?$AAa?$AAc?$AAk?$AA?$AA@ 10011330     wmstub:drmauth.obj
 0003:00000344       ??_C@_1BM@LAJH@?$AAW?$AAM?$AA?1?$AAA?$AAl?$AAb?$AAu?$AAm?$AAT?$AAi?$AAt?$AAl?$AAe?$AA?$AA@ 10011344     wmstub:drmauth.obj
 0003:00000360       ??_C@_1BE@NMAK@?$AAD?$AAR?$AAM?$AA_?$AAL?$AAe?$AAv?$AAe?$AAl?$AA?$AA@ 10011360     wmstub:drmauth.obj
 0003:00000374       ??_C@_1BE@OCCE@?$AAD?$AAR?$AAM?$AA_?$AAF?$AAl?$AAa?$AAg?$AAs?$AA?$AA@ 10011374     wmstub:drmauth.obj
 0003:00000388       ??_C@_1BA@NLDB@?$AAU?$AAs?$AAe?$AA_?$AAD?$AAR?$AAM?$AA?$AA@ 10011388     wmstub:drmauth.obj
 0003:00000398       ??_C@_1BE@JCKD@?$AAC?$AAo?$AAp?$AAy?$AAr?$AAi?$AAg?$AAh?$AAt?$AA?$AA@ 10011398     wmstub:drmauth.obj
 0003:000003ac       ??_C@_1O@JJKF@?$AAR?$AAa?$AAt?$AAi?$AAn?$AAg?$AA?$AA@ 100113ac     wmstub:drmauth.obj
 0003:000003bc       ??_C@_1BI@CNDL@?$AAD?$AAe?$AAs?$AAc?$AAr?$AAi?$AAp?$AAt?$AAi?$AAo?$AAn?$AA?$AA@ 100113bc     wmstub:drmauth.obj
 0003:000003d4       ??_C@_1O@MLJI@?$AAA?$AAu?$AAt?$AAh?$AAo?$AAr?$AA?$AA@ 100113d4     wmstub:drmauth.obj
 0003:000003e4       ??_C@_1M@NPJG@?$AAT?$AAi?$AAt?$AAl?$AAe?$AA?$AA@ 100113e4     wmstub:drmauth.obj
 0003:000003f0       ??_C@_1BO@MNPK@?$AAO?$AAp?$AAt?$AAi?$AAm?$AAa?$AAl?$AAB?$AAi?$AAt?$AAr?$AAa?$AAt?$AAe?$AA?$AA@ 100113f0     wmstub:drmauth.obj
 0003:00000410       ??_C@_1BO@OHF@?$AAC?$AAu?$AAr?$AAr?$AAe?$AAn?$AAt?$AAB?$AAi?$AAt?$AAr?$AAa?$AAt?$AAe?$AA?$AA@ 10011410     wmstub:drmauth.obj
 0003:00000430       ??_C@_1BC@HCCL@?$AAH?$AAa?$AAs?$AAV?$AAi?$AAd?$AAe?$AAo?$AA?$AA@ 10011430     wmstub:drmauth.obj
 0003:00000444       ??_C@_1BE@BING@?$AAH?$AAa?$AAs?$AAS?$AAc?$AAr?$AAi?$AAp?$AAt?$AA?$AA@ 10011444     wmstub:drmauth.obj
 0003:00000458       ??_C@_1BC@PCDH@?$AAH?$AAa?$AAs?$AAI?$AAm?$AAa?$AAg?$AAe?$AA?$AA@ 10011458     wmstub:drmauth.obj
 0003:0000046c       ??_C@_1BC@PBCE@?$AAH?$AAa?$AAs?$AAA?$AAu?$AAd?$AAi?$AAo?$AA?$AA@ 1001146c     wmstub:drmauth.obj
 0003:00000480       ??_C@_1BO@CDJH@?$AAS?$AAi?$AAg?$AAn?$AAa?$AAt?$AAu?$AAr?$AAe?$AA_?$AAN?$AAa?$AAm?$AAe?$AA?$AA@ 10011480     wmstub:drmauth.obj
 0003:000004a0       ??_C@_1BG@OOHP@?$AAI?$AAs?$AA_?$AAT?$AAr?$AAu?$AAs?$AAt?$AAe?$AAd?$AA?$AA@ 100114a0     wmstub:drmauth.obj
 0003:000004b8       ??_C@_1BK@JHKK@?$AAI?$AAs?$AA_?$AAP?$AAr?$AAo?$AAt?$AAe?$AAc?$AAt?$AAe?$AAd?$AA?$AA@ 100114b8     wmstub:drmauth.obj
 0003:000004d4       ??_C@_1BE@BLF@?$AAB?$AAr?$AAo?$AAa?$AAd?$AAc?$AAa?$AAs?$AAt?$AA?$AA@ 100114d4     wmstub:drmauth.obj
 0003:000004e8       ??_C@_1BE@LNKF@?$AAS?$AAt?$AAr?$AAi?$AAd?$AAa?$AAb?$AAl?$AAe?$AA?$AA@ 100114e8     wmstub:drmauth.obj
 0003:000004fc       ??_C@_1BC@PLAJ@?$AAS?$AAe?$AAe?$AAk?$AAa?$AAb?$AAl?$AAe?$AA?$AA@ 100114fc     wmstub:drmauth.obj
 0003:00000510       ??_C@_1BA@BAC@?$AAB?$AAi?$AAt?$AAr?$AAa?$AAt?$AAe?$AA?$AA@ 10011510     wmstub:drmauth.obj
 0003:00000520       ??_C@_1BC@BAFD@?$AAD?$AAu?$AAr?$AAa?$AAt?$AAi?$AAo?$AAn?$AA?$AA@ 10011520     wmstub:drmauth.obj
 0003:00000538       ?g_cWMSDKCerts@@3KA        10011538     wmstub:certkeys.obj
 0003:00000540       ?g_rgWMSDKCerts@@3PAUCERT_PAIR@@A 10011540     wmstub:certkeys.obj
 0003:00000838       _vmulnn                    10011838     wmstub:vmul.obj
 0003:00000870       __fltused                  10011870     MSVCRT:fltused.obj
 0003:00000880       ___scrt_native_dllmain_reason 10011880     MSVCRT:utility.obj
 0003:00000890       ___isa_enabled             10011890     MSVCRT:_cpu_disp_.obj
 0003:00000894       ___security_cookie_complement 10011894     MSVCRT:gs_cookie.obj
 0003:00000898       ___security_cookie         10011898     MSVCRT:gs_cookie.obj
 0003:0000089c       ___scrt_ucrt_dll_is_in_use 1001189c     MSVCRT:ucrt_stubs.obj
 0003:000008a0       ??_R0?AVbad_alloc@std@@@8  100118a0     MSVCRT:throw_bad_alloc.obj
 0003:000008bc       ??_R0?AVexception@std@@@8  100118bc     MSVCRT:throw_bad_alloc.obj
 0003:000008d8       ??_R0?AVbad_array_new_length@std@@@8 100118d8     MSVCRT:throw_bad_alloc.obj
 0003:00000900       ??_R0?AVtype_info@@@8      10011900     MSVCRT:std_type_info_static.obj
 0003:00000918       ?gCritSect@@3U_RTL_CRITICAL_SECTION@@A 10011918     wmstub:pkcrypto.obj
 0003:00000930       ?gCritSectInited@@3HA      10011930     wmstub:pkcrypto.obj
 0003:00000934       _mp_errno                  10011934     wmstub:mpglobal.obj
 0003:00000e24       ____NtQuerySystemInformationRNG 10011e24     wmstub:randlib.obj
 0003:00000e28       ____NtOpenFileRNG          10011e28     wmstub:randlib.obj
 0003:00000e2c       ____RtlInitUnicodeStringRNG 10011e2c     wmstub:randlib.obj
 0003:00000e30       ____GetCursorPosRNG        10011e30     wmstub:randlib.obj
 0003:00000e34       ____GetMessageTimeRNG      10011e34     wmstub:randlib.obj
 0003:00000e48       ___scrt_current_native_startup_state 10011e48     MSVCRT:utility.obj
 0003:00000e4c       ___scrt_native_startup_lock 10011e4c     MSVCRT:utility.obj
 0003:00000e70       ?__type_info_root_node@@3U__type_info_node@@A 10011e70     MSVCRT:tncleanup.obj
 0003:00000e78       ?_OptionsStorage@?1??__local_stdio_printf_options@@9@4_KA 10011e78     MSVCRT:default_local_stdio_options.obj
 0003:00000e80       ?_OptionsStorage@?1??__local_stdio_scanf_options@@9@4_KA 10011e80     MSVCRT:default_local_stdio_options.obj
 0003:00000e88       ___scrt_debugger_hook_flag 10011e88     MSVCRT:utility_desktop.obj
 0003:00000e8c       ___isa_available           10011e8c     MSVCRT:_cpu_disp_.obj
 0003:00000e90       ___favor                   10011e90     MSVCRT:_cpu_disp_.obj
 0003:000011b4       ___dyn_tls_init_callback   100121b4     <common>

 entry point at        0001:0000d305

 Static symbols

 0002:ffff1000       .idata$6                   10000000     ucrt:api-ms-win-crt-math-l1-1-0.dll
 0001:000004d0       ?dw_to_modular@@YGHPBKKPA_IPBUmp_modulus_t@@@Z 100014d0 f   wmstub:pkcrypto.obj
 0001:000005d0       ?ec_init@@YGJPAUPK_DATA@@PBK11111@Z 100015d0 f   wmstub:pkcrypto.obj
 0001:000007c0       ?my_ecaffine_exponentiation@@YGHPB_IQB_IKPA_IPAUecurve_t@@@Z 100017c0 f   wmstub:pkcrypto.obj
 0001:00000a40       ?fast_ecaffine_exponentiation@@YGHPB_IQB_IKPA_IPAUecurve_t@@@Z 10001a40 f   wmstub:pkcrypto.obj
 0001:00000c60       ?ecaffine_to_dwords@@YGHPA_IPAKPBUecurve_t@@@Z 10001c60 f   wmstub:pkcrypto.obj
 0001:00002a10       _to_kara2@16               10003a10 f   wmstub:modular.obj
 0001:00003e00       _ec_concurrent_operations@4 10004e00 f   wmstub:ecexpon.obj
 0001:00004600       _affine_insert_bucket@16   10005600 f   wmstub:ecexpon.obj
 0001:000046f0       _proj5_insert_bucket@16    100056f0 f   wmstub:ecexpon.obj
 0001:000047d0       _get_ec_concurrent_slot@4  100057d0 f   wmstub:ecexpon.obj
 0001:00004810       _ecaffine_to_ecproj5@16    10005810 f   wmstub:ecexpon.obj
 0001:000048a0       _ecproj5_add_ecaffine@20   100058a0 f   wmstub:ecexpon.obj
 0001:000048f0       _ecproj5_add_ecproj5@20    100058f0 f   wmstub:ecexpon.obj
 0001:00004e70       _ecproj5_doubling@16       10005e70 f   wmstub:ecexpon.obj
 0001:000051d0       _ecproj5_set_infinite@12   100061d0 f   wmstub:ecexpon.obj
 0001:00005230       _ecproj5_to_ecaffine@16    10006230 f   wmstub:ecexpon.obj
 0001:000052e0       _schedule_affine_add_and_sub@20 100062e0 f   wmstub:ecexpon.obj
 0001:000053c0       _schedule_affine_add_or_sub@20 100063c0 f   wmstub:ecexpon.obj
 0001:00008580       _kara_merge@24             10009580 f   wmstub:kara.obj
 0001:00008d00       _kara_difs@20              10009d00 f   wmstub:kara.obj
 0001:00008fe1       invert_endian_input        10009fe1 f   wmstub:shafast.obj
 0001:00009010       expand_loop                1000a010 f   wmstub:shafast.obj
 0001:00009b65       expand_loop2               1000ab65 f   wmstub:shafast.obj
 0001:0000b120       _vmul11_c@16               1000c120 f   wmstub:vmul.obj
 0001:0000b1a0       _vmul22_c@16               1000c1a0 f   wmstub:vmul.obj
 0001:0000b340       _vmul33_asm@16             1000c340 f   wmstub:vmul.obj
 0001:0000b5c0       _vmul44_asm@16             1000c5c0 f   wmstub:vmul.obj
 0001:0000bab0       _vmul66_asm@16             1000cab0 f   wmstub:vmul.obj
 0001:0000bd80       _vmul88_asm@16             1000cd80 f   wmstub:vmul.obj
 0001:0000c0a0       _vmul1212_asm@16           1000d0a0 f   wmstub:vmul.obj
 0001:0000c6b4       rc4_loop                   1000d6b4 f   wmstub:rc4fast.obj
 0001:0000c6df       rc4_done                   1000d6df f   wmstub:rc4fast.obj
 0001:0000c705       init_loop                  1000d705 f   wmstub:rc4fast.obj
 0001:0000c728       permute_loop               1000d728 f   wmstub:rc4fast.obj
 0001:0000c74b       skip_zero_k                1000d74b f   wmstub:rc4fast.obj
 0001:0000cffd       ?dllmain_crt_dispatch@@YGHQAUHINSTANCE__@@KQAX@Z 1000dffd f   MSVCRT:dll_dllmain.obj
 0001:0000d050       ?dllmain_crt_process_attach@@YAHQAUHINSTANCE__@@QAX@Z 1000e050 f   MSVCRT:dll_dllmain.obj
 0001:0000d162       ?dllmain_crt_process_detach@@YAH_N@Z 1000e162 f   MSVCRT:dll_dllmain.obj
 0001:0000d1df       ?dllmain_dispatch@@YAHQAUHINSTANCE__@@KQAX@Z 1000e1df f   MSVCRT:dll_dllmain.obj
 0001:0000d2db       ?dllmain_raw@@YGHQAUHINSTANCE__@@KQAX@Z 1000e2db f   MSVCRT:dll_dllmain.obj
 0001:0000d360       $$000000                   1000e360     MSVCRT:ulldiv.obj
 0001:0000d3d0       $$000000                   1000e3d0     MSVCRT:chkstk.obj
 0001:0000d400       $$000000                   1000e400     MSVCRT:llmul.obj
 0001:0000d440       ?find_pe_section@@YAPAU_IMAGE_SECTION_HEADER@@QAEI@Z 1000e440 f   MSVCRT:utility.obj
 0001:0000d9d0       $$000000                   1000e9d0     MSVCRT:_sehprolg4_.obj
 0002:00000120       $SG91573                   1000f120     wmstubber.obj
 0002:00000134       $SG91575                   1000f134     wmstubber.obj
 0002:00000144       $SG91577                   1000f144     wmstubber.obj
 0002:00000158       $SG91579                   1000f158     wmstubber.obj
 0002:0000016c       $SG91581                   1000f16c     wmstubber.obj
 0002:00000180       $SG91583                   1000f180     wmstubber.obj
 0002:0000019c       $SG91585                   1000f19c     wmstubber.obj
 0002:000001b4       $SG91587                   1000f1b4     wmstubber.obj
 0002:000001d4       $SG91589                   1000f1d4     wmstubber.obj
 0002:000001e8       $SG91591                   1000f1e8     wmstubber.obj
 0002:000001fc       $SG91593                   1000f1fc     wmstubber.obj
 0002:00000210       $SG91595                   1000f210     wmstubber.obj
 0002:00000224       $SG91597                   1000f224     wmstubber.obj
 0002:00000244       $SG91599                   1000f244     wmstubber.obj
 0002:00000264       $SG91602                   1000f264     wmstubber.obj
 0002:00000270       $SG91604                   1000f270     wmstubber.obj
 0002:00000280       $SG91606                   1000f280     wmstubber.obj
 0002:00000298       $SG91608                   1000f298     wmstubber.obj
 0002:000002a8       $SG91610                   1000f2a8     wmstubber.obj
 0002:000002bc       $SG91612                   1000f2bc     wmstubber.obj
 0002:000002cc       $SG91614                   1000f2cc     wmstubber.obj
 0002:000002e0       $SG91616                   1000f2e0     wmstubber.obj
 0002:000002f4       $SG91618                   1000f2f4     wmstubber.obj
 0002:00000310       $SG91620                   1000f310     wmstubber.obj
 0002:00000324       $SG91622                   1000f324     wmstubber.obj
 0002:00000344       $SG91624                   1000f344     wmstubber.obj
 0002:00000368       $SG91626                   1000f368     wmstubber.obj
 0002:0000037c       $SG91628                   1000f37c     wmstubber.obj
 0002:0000038c       $SG91630                   1000f38c     wmstubber.obj
 0002:000003a4       $SG91632                   1000f3a4     wmstubber.obj
 0002:000003b4       $SG91634                   1000f3b4     wmstubber.obj
 0002:000003d4       $SG91636                   1000f3d4     wmstubber.obj
 0002:000003f4       $SG91638                   1000f3f4     wmstubber.obj
 0002:00000414       $SG91640                   1000f414     wmstubber.obj
 0002:00000430       $SG91643                   1000f430     wmstubber.obj
 0002:00000444       $SG91645                   1000f444     wmstubber.obj
 0002:0000045c       $SG91647                   1000f45c     wmstubber.obj
 0002:00000470       $SG91649                   1000f470     wmstubber.obj
 0002:00000484       $SG91651                   1000f484     wmstubber.obj
 0002:000004a4       $SG91653                   1000f4a4     wmstubber.obj
 0002:000004c8       $SG91655                   1000f4c8     wmstubber.obj
 0002:000004ec       $SG91657                   1000f4ec     wmstubber.obj
 0002:00000514       $SG91659                   1000f514     wmstubber.obj
 0002:00000534       $SG91661                   1000f534     wmstubber.obj
 0002:00000558       $SG91663                   1000f558     wmstubber.obj
 0002:00000578       $SG91665                   1000f578     wmstubber.obj
 0002:000005c8       _ecdw_q                    1000f5c8     wmstub:pkcrypto.obj
 0002:000005dc       _ecdw_order                1000f5dc     wmstub:pkcrypto.obj
 0002:000005f0       _ecdw_a                    1000f5f0     wmstub:pkcrypto.obj
 0002:00000604       _ecdw_b                    1000f604     wmstub:pkcrypto.obj
 0002:00000618       _ecdw_genx                 1000f618     wmstub:pkcrypto.obj
 0002:0000062c       _ecdw_geny                 1000f62c     wmstub:pkcrypto.obj
 0002:00000680       _random_multiplier         1000f680     wmstub:randsupp.obj
 0002:00000758       _PADDING$S9593             1000f758     wmstub:md4ms.obj
 0002:00000804       _GS_ExceptionPointers      1000f804     MSVCRT:gs_report.obj
 0002:00000c30       __sehtable$?dllmain_crt_process_attach@@YAHQAUHINSTANCE__@@QAX@Z 1000fc30     MSVCRT:dll_dllmain.obj
 0002:00000c50       __sehtable$?dllmain_crt_process_detach@@YAH_N@Z 1000fc50     MSVCRT:dll_dllmain.obj
 0002:00000c70       __sehtable$?dllmain_dispatch@@YAHQAUHINSTANCE__@@KQAX@Z 1000fc70     MSVCRT:dll_dllmain.obj
 0002:00000c90       __sehtable$___scrt_is_nonwritable_in_current_image 1000fc90     MSVCRT:utility.obj
 0002:00000d40       .edata                     1000fd40     wmstubber.exp
 0002:00000d68       rgpv                       1000fd68     wmstubber.exp
 0002:00000d6c       rgszName                   1000fd6c     wmstubber.exp
 0002:00000d70       rgwOrd                     1000fd70     wmstubber.exp
 0002:00000d72       szName                     1000fd72     wmstubber.exp
 0002:00000d80       $N00001                    1000fd80     wmstubber.exp
 0002:00000fb0       .idata$6                   1000ffb0     vcruntime:VCRUNTIME140.dll
 0002:000010b0       .idata$6                   100100b0     ucrt:api-ms-win-crt-runtime-l1-1-0.dll
 0002:000010d2       .idata$6                   100100d2     ucrt:api-ms-win-crt-heap-l1-1-0.dll
 0002:00001364       .idata$6                   10010364     kernel32:KERNEL32.dll
 0002:000013c8       .idata$6                   100103c8     advapi32:ADVAPI32.dll
 0002:000013f8       .idata$6                   100103f8     ole32:ole32.dll
 0003:00000000       _g_wszWMDuration           10011000     wmstub:drmauth.obj
 0003:00000004       _g_wszWMBitrate            10011004     wmstub:drmauth.obj
 0003:00000008       _g_wszWMSeekable           10011008     wmstub:drmauth.obj
 0003:0000000c       _g_wszWMStridable          1001100c     wmstub:drmauth.obj
 0003:00000010       _g_wszWMBroadcast          10011010     wmstub:drmauth.obj
 0003:00000014       _g_wszWMProtected          10011014     wmstub:drmauth.obj
 0003:00000018       _g_wszWMTrusted            10011018     wmstub:drmauth.obj
 0003:0000001c       _g_wszWMSignature_Name     1001101c     wmstub:drmauth.obj
 0003:00000020       _g_wszWMHasAudio           10011020     wmstub:drmauth.obj
 0003:00000024       _g_wszWMHasImage           10011024     wmstub:drmauth.obj
 0003:00000028       _g_wszWMHasScript          10011028     wmstub:drmauth.obj
 0003:0000002c       _g_wszWMHasVideo           1001102c     wmstub:drmauth.obj
 0003:00000030       _g_wszWMCurrentBitrate     10011030     wmstub:drmauth.obj
 0003:00000034       _g_wszWMOptimalBitrate     10011034     wmstub:drmauth.obj
 0003:00000038       _g_wszWMTitle              10011038     wmstub:drmauth.obj
 0003:0000003c       _g_wszWMAuthor             1001103c     wmstub:drmauth.obj
 0003:00000040       _g_wszWMDescription        10011040     wmstub:drmauth.obj
 0003:00000044       _g_wszWMRating             10011044     wmstub:drmauth.obj
 0003:00000048       _g_wszWMCopyright          10011048     wmstub:drmauth.obj
 0003:0000004c       _g_wszWMUse_DRM            1001104c     wmstub:drmauth.obj
 0003:00000050       _g_wszWMDRM_Flags          10011050     wmstub:drmauth.obj
 0003:00000054       _g_wszWMDRM_Level          10011054     wmstub:drmauth.obj
 0003:00000058       _g_wszWMAlbumTitle         10011058     wmstub:drmauth.obj
 0003:0000005c       _g_wszWMTrack              1001105c     wmstub:drmauth.obj
 0003:00000060       _g_wszWMPromotionURL       10011060     wmstub:drmauth.obj
 0003:00000064       _g_wszWMAlbumCoverURL      10011064     wmstub:drmauth.obj
 0003:00000068       _g_wszWMGenre              10011068     wmstub:drmauth.obj
 0003:0000006c       _g_wszWMYear               1001106c     wmstub:drmauth.obj
 0003:00000070       _g_wszWMGenreID            10011070     wmstub:drmauth.obj
 0003:00000074       _g_wszWMMCDI               10011074     wmstub:drmauth.obj
 0003:00000078       _g_wszWMBannerImageType    10011078     wmstub:drmauth.obj
 0003:0000007c       _g_wszWMBannerImageData    1001107c     wmstub:drmauth.obj
 0003:00000080       _g_wszWMBannerImageURL     10011080     wmstub:drmauth.obj
 0003:00000084       _g_wszWMCopyrightURL       10011084     wmstub:drmauth.obj
 0003:00000088       _g_wszWMNSCName            10011088     wmstub:drmauth.obj
 0003:0000008c       _g_wszWMNSCAddress         1001108c     wmstub:drmauth.obj
 0003:00000090       _g_wszWMNSCPhone           10011090     wmstub:drmauth.obj
 0003:00000094       _g_wszWMNSCEmail           10011094     wmstub:drmauth.obj
 0003:00000098       _g_wszWMNSCDescription     10011098     wmstub:drmauth.obj
 0003:0000009c       _g_wszEarlyDataDelivery    1001109c     wmstub:drmauth.obj
 0003:000000a0       _g_wszJustInTimeDecode     100110a0     wmstub:drmauth.obj
 0003:000000a4       _g_wszSingleOutputBuffer   100110a4     wmstub:drmauth.obj
 0003:000000a8       _g_wszSoftwareScaling      100110a8     wmstub:drmauth.obj
 0003:000000ac       _g_wszDeliverOnReceive     100110ac     wmstub:drmauth.obj
 0003:000000b0       _g_wszDeinterlaceMode      100110b0     wmstub:drmauth.obj
 0003:000000b4       _g_wszOriginalSourceFormatTag 100110b4     wmstub:drmauth.obj
 0003:00000720       _random_seed               10011720     wmstub:randsupp.obj
 0003:00000728       _g_dwRC4RekeyParam$S16227  10011728     wmstub:randlib.obj
 0003:0000072c       _?g_dwRC4BytesUsed@?1??RandomFillBuffer@@9@9$S16326 1001172c     wmstub:randlib.obj
 0003:00000730       _?fIsWinNT@?1??IsRNGWinNT@@9@9$S16467 10011730     wmstub:randlib.obj
 0003:00000738       _vmul_flt                  10011738     wmstub:vmul.obj
 0003:00000938       _active_allocs             10011938     wmstub:mpglobal.obj
 0003:00000940       _paddings                  10011940     wmstub:kara.obj
 0003:00000a90       _?dwUserNameSize@?BE@??GatherRandomKey@@9@9$S16378 10011a90     wmstub:randlib.obj
 0003:00000a98       _g_VeryLargeHash$S16229    10011a98     wmstub:randlib.obj
 0003:00000ae8       _?g_rc4key@?1??RandomFillBuffer@@9@9$S16324 10011ae8     wmstub:randlib.obj
 0003:00000bec       _?dwComputerNameSize@?BE@??GatherRandomKey@@9@9$S16376 10011bec     wmstub:randlib.obj
 0003:00000bf0       _g_CircularHashCtx$S16228  10011bf0     wmstub:randlib.obj
 0003:00000d10       _?lpComputerName@?BE@??GatherRandomKey@@9@9$S16380 10011d10     wmstub:randlib.obj
 0003:00000d20       _?lpUserName@?BE@??GatherRandomKey@@9@9$S16382 10011d20     wmstub:randlib.obj
 0003:00000e38       _?fInitialized@?1??InitRand@@9@9$S16296 10011e38     wmstub:randlib.obj
 0003:00000e3c       _?fIKnow@?1??IsRNGWinNT@@9@9$S16465 10011e3c     wmstub:randlib.obj
 0003:00000e40       _?dwCounterType@?1??GatherCPUSpecificCountersPrivileged@@9@9$S14600 10011e40     wmstub:cpu.obj
 0003:00000e44       ?__proc_attached@@3HA      10011e44     MSVCRT:dll_dllmain.obj
 0003:00000e50       ?module_local_atexit_table@@3U_onexit_table_t@@A 10011e50     MSVCRT:utility.obj
 0003:00000e5c       ?module_local_at_quick_exit_table@@3U_onexit_table_t@@A 10011e5c     MSVCRT:utility.obj
 0003:00000e68       ?is_initialized_as_dll@@3_NA 10011e68     MSVCRT:utility.obj
 0003:00000e98       _GS_ExceptionRecord        10011e98     MSVCRT:gs_report.obj
 0003:00000ee8       _GS_ContextRecord          10011ee8     MSVCRT:gs_report.obj
 0004:00000000       __guard_fids_?dllmain_crt_process_attach@@YAHQAUHINSTANCE__@@QAX@Z 10013000     MSVCRT:dll_dllmain.obj
 0004:00000008       __guard_fids_?dllmain_dispatch@@YAHQAUHINSTANCE__@@KQAX@Z 10013008     MSVCRT:dll_dllmain.obj
 0004:0000000c       __guard_fids___except_handler4 1001300c     MSVCRT:_chandler4gs_.obj
 0004:00000010       __guard_fids__             10013010     MSVCRT:throw_bad_alloc.obj
 0004:00000018       __guard_fids__             10013018     MSVCRT:throw_bad_alloc.obj
 0004:00000020       __guard_fids__             10013020     MSVCRT:throw_bad_alloc.obj
 0004:00000028       __guard_fids__             10013028     MSVCRT:throw_bad_alloc.obj
 0004:0000002c       __guard_fids__             1001302c     MSVCRT:throw_bad_alloc.obj
 0004:00000030       __guard_fids__             10013030     MSVCRT:throw_bad_alloc.obj
 0004:00000034       __guard_fids__             10013034     MSVCRT:throw_bad_alloc.obj
 0004:00000038       __guard_fids__             10013038     MSVCRT:throw_bad_alloc.obj
 0004:0000003c       __guard_fids__             1001303c     MSVCRT:guard_support.obj
 0004:00000040       __guard_fids__             10013040     MSVCRT:std_type_info_static.obj
 0005:000000a0       $R000000                   100140a0     wmstubber_res.res
 0005:000004a8       $R000408                   100144a8     wmstubber_res.res

 Exports

  ordinal    name

        1    _get_wmcreatecertificate_func
               exported name: get_wmcreatecertificate_func
